:020000003328A3
:020008006D2861
:10002000820741344D345034203448344F345534F1
:100030005234533420342B3431343234333420347A
:100040002034003441344D3450342B343934393475
:100050003934203420345634383438342E3438345B
:10006000203420340034C220FD218B128B17F53050
:10007000C8008101FA30B2008316823081008312F9
:10008000051840284D10CD14C901CA0193018B12E7
:10009000051C48280508960081018B16CD14000028
:1000A000000000000000051C5928C90F4E28CA0A8C
:1000B0004E2849084A0403194E284908CB004A082B
:1000C000CC00961C6528131066281314C901CA01B8
:1000D000CD104D1C68289B2240280B11C80B09002D
:1000E000F530C800CD188B284D148B129520433065
:1000F0009A00CA20D5200921C821B01B82282B30A4
:10010000B30084282D30B300ED210A309A00CA20B4
:100110004D149B2209002030B3003030B400B500EC
:10012000B60043309A00CA2088286E224B08A400EB
:100130004C08A300AC201C2120089200210891004B
:1001400022089000C821131CA8282B30B300AA282D
:100150002D30B300ED21080000308900831608140B
:1001600083120808A0000130890083160814831246
:100170000808A100023089008316081483120808B9
:10018000A20008001030840000308000840A841F20
:10019000C52808001A0830223308452234084522B1
:1001A000350845223608452208003208A2003108E9
:1001B000A1003008A0001008A5001108A400120832
:1001C000A300131CF920EB202208B2002108B10083
:1001D0002008B00008002508A207031CF228A10A85
:1001E0000319A00A2408A1070318A00A2308A007DE
:1001F0000800A509A50A0319A403A4090319A30368
:10020000A3090800A209A20A0319A103A109A009D0
:10021000080093133008A0003108A1003208A200A2
:10022000A01F1429931702211130A3009430A400B9
:100230001C21931B02210800A601A701A801200D83
:10024000A70D2408A7022308031C230FA6020301FD
:10025000031C0130A802A00D0730A900200DA70D36
:10026000A60DA80D2408201C3F29A7022308031C63
:10027000230FA6020301031C0130A8024829A70787
:1002800023080318230FA607030103180130A8074A
:10029000A00DA90B2E29210DA70DA60DA80D240830
:1002A000201C5C29A7022308031C230FA6020301BC
:1002B000031C0130A8026529A70723080318230F90
:1002C000A607030103180130A807A10D0730A900F4
:1002D000210DA70DA60DA80D2408211C7929A70220
:1002E0002308031C230FA6020301031C0130A802EC
:1002F0008229A70723080318230FA6070301031861
:100300000130A807A10DA90B6829220DA70DA60D84
:10031000A80D2408211C9629A7022308031C230FDB
:10032000A6020301031C0130A8029F29A707230886
:100330000318230FA607030103180130A807A20D15
:100340000730A900220DA70DA60DA80D2408221C18
:10035000B329A7022308031C230FA6020301031CD1
:100360000130A802BC29A70723080318230FA607FA
:10037000030103180130A807A20DA90BA229221816
:10038000C7292408A70723080318230FA607080076
:10039000A01B022103101030C500C201C301C4011B
:1003A000A20DA10DC40DC30DC20DC50BD8290800A7
:1003B00044308400E22143308400E2214230840052
:1003C000E221D029033000079A009A1980003030CA
:1003D00000079A009A1B80000800B601B501B4011D
:1003E00044080F39303EB600440E0F39303EB50098
:1003F00043080F39303EB4000800831603308500EF
:100400000F3086008312850186011E305F2205169B
:1004100030308600051210305F220516303086001D
:10042000051210305F22051630308600051210309C
:100430005F22051620308600051210305F2228301A
:1004400033220C303322013033221C30332200306F
:100450003022003064224030302211306422080003
:10046000803833220800AA0010305F228511051160
:1004700005162A088600051210305F2205162A0E7E
:10048000860010305F2205120800AA0010305F229B
:100490008511051505162A088600051210305F2201
:1004A00005162A0E860010305F2205120800023061
:1004B00033220800A530AD00AD0B5C2A0800AE0069
:1004C0005A22AE0B602A0800AB001020FF39031936
:1004D0006D2A45222B08013E642A080006198A2A43
:1004E0004B08A5004C08A4000030A3000A308F0080
:1004F000EB208F0B782A20088800003089008B229F
:1005000021088800013089008B22220888000230EF
:1005100089008B22080083168B130815553089003B
:10052000AA308900881408118818942A08128312A6
:100530008B178B1308008B130330A0003A30A100F7
:100540009030A200C0224A08A3004908A4001C2140
:100550002008BB002108BC002208BD000030A30019
:100560000A30A4001C21C821ED213408B30035084D
:10057000B4002E30B5004A309A00CA208B1708000C
:10058000C901CA018619C22A00000000000000004B
:100590000000861DC92A0000861DD22AC90FCC2A58
:0605A000CA0ACC2A080083
:0642000000001E0000009A
:00000001FF
